:020000040000FA
:020000000828CE
:08000800B92CC02A8A01820014
:10001000FF30A200FF30A300DF220A300B2425129C
:100020005F240330D622323024240330D6223230EB
:1000300024240330D622323024243230CA222830FD
:10004000CA2276225A22742222118124A3177C24E8
:10005000A3167E2423177D24A6010230A700A80141
:100060000230A90007309F00B022B901A011BA01E7
:10007000BB01061F3F28BE30B700B80190210630F3
:10008000B400D630B3000830B6007030B500241587
:100090006124B022C8210230FD23B02280213B0818
:1000A000643C03185428BB012B303B02031C592825
:1000B0003D24BB0A902107211521342179219C215F
:1000C000861A6E28861B6E28061F6E28B90A013014
:1000D000042402303902031C6E28B901B908031D3B
:1000E0008228A01D74287921A011A012BA01861EB1
:1000F0007B2824156124861F7F2824116124201A5F
:1001000082289C213908013C031DC1282415612443
:10011000A01990286130BD00CE30BE001030EC2117
:1001200001300B240330A8225330C2226530C22292
:100130007430C2222030C222861AA028861FA82826
:10014000BA0A28303A02031CA8282830BA00A016A0
:10015000861AAE28861BAE28A012BA01861EB428C5
:10016000A01EB428F620B528E720861FBB28A01EB5
:10017000BB28D220BC28C3203421A0152012013076
:100180000B246028C228290828020318D028861FBB
:10019000D028A80A28082902031DCF28D220D12858
:1001A000A801080015212019E6283808BC003708E6
:1001B000BD00BE010130BF0012234008B800410855
:1001C000B7002013A01FE5282017072108002708E3
:1001D00026020318F428861EF428A60A26082702F9
:1001E000031DF328F620F528A60108001521A01804
:1001F00006293808BC003708BD00BE010130BF0029
:1002000080234008B8004108B700072108003408DF
:10021000BC003308BD003808BE003708BF0080238B
:100220004008AB004108AA00080036082B02031C56
:10023000232935082A02031C2329A0143608AB0001
:100240003508AA002429A0102B083402031C3229E7
:100250002A083302031C322920153408AB00330866
:10026000AA003329201108002A08B1002B08B20087
:100270003108BC003208BD001430BE00BF01EB22C3
:100280003C08B1003D08B2004008AC004108AD0098
:100290002D08BF002C087E223C08AE003D08AF00B0
:1002A0003E08B0000030AC220430BC002F08BD0076
:1002B000203094230430BC003008BD0030309F2330
:1002C0002E30C2220430BC003108C0000530C1000D
:1002D000AA244208BF003F08BD003030B3232030BD
:1002E000C2224D30C2220030A8224830C2227A30C9
:1002F000C22A90216130BD002B08BE002A08EC29DB
:100300000130BC0055243D08B7000230BC00552424
:100310003D08B8000330BC0055243D08BB00080070
:100320000130BC0037083F240230BC0038083F24AD
:100330000330BC003B083F2C6130BD00F6213E0875
:10034000BC003C1BB4290330A8224230C2227530C5
:10035000C2227330C2227930C22220126130BD0025
:10036000CE30BE000030EC213C1FC7290330A8224C
:100370004C30C2226F30C2226330C2226B30C222A4
:1003800020166130BD00CE30BE002430EC210800C4
:100390000030AC222030C2224630C2224D30C22270
:1003A0002030C2225430C2227230C2226130C222B6
:1003B0006E30C2220030A8227330C2226D30C222B9
:1003C0006930C2227430C2227430C2226530C22227
:1003D0007230C2222030C22ABF003D08FD213E08F3
:1003E000172228223F08172228225A2ABE003D0839
:1003F00003220A223F08BE00242AC00067220310FD
:10040000400D1722282ABF00672203103F0D013E2E
:100410001722282ABF000830C0000310BF0D362263
:100420003F10A01F142A3F14C00B0D2A0800C10062
:100430000830C200A013C11F1E2AA01749220310B2
:10044000C10DC20B1A2A080026225A2AA013492AD3
:100450007422A21482247422221483247422051884
:10046000322A2F2A742222108324742A7422A2147E
:10047000822474222214832474220518402A3D2ADF
:100480007422A013851C452AA017742222108324ED
:10049000742A7422A210A01F4E2AA214822474224D
:1004A0002214832474220518562A532A74222210F7
:1004B0008324742A7422A21082247422221083249A
:1004C0007422221483247422A2148224742A742293
:1004D000A21482247422221483247422A21082245F
:1004E000742222108324742A0C30302C24106324AC
:1004F00022108324A4106224A210822CC000BC010C
:10050000BD01BE011030C1003E0898224208BE0065
:100510003D0898224208BD003C0898224208BC00D1
:10052000C00DBF0DBE0DBD0DBC0DC10B842A080052
:10053000C2004208033EC300C31DA02A4308C200F4
:100540004208303EC300C31FA72A4308C200080068
:10055000BD003D08C03ECA2ABC003C08803ECA2AF5
:100560000830CA220130CA22C83024240230CA22EC
:10057000C83024240630CA220C30CA22C830242CA9
:100580002108C400C40025165F24440E0F39D6226A
:100590004408D62ABE0025125F243E0E0F39D6220B
:1005A000823024243E08D6228230242CC500A41593
:1005B000602445086424A4116024FA30302C0030F3
:1005C000642425125F24A4116024003073242312B4
:1005D0007F24A211802CC100C001C1010130C200E2
:1005E000C301BF1BF92A0310C20DC30DBE0DBF0D01
:1005F000F12A3E083C02C4000030031C01303F07D2
:100600003D02031C0A2BBD004408BC004208C00781
:100610004308C1070310BF0CBE0CC30CC20C031C63
:10062000F92A08003C083E020318392BA0173D08A0
:100630003F020318222B3E083C02C0003F083D0247
:10064000C100382B3D083F02031D2B2B3E083C0206
:10065000C000C101382B3F083D020318382B3E086B
:100660003C02C20001304202C0003F083D02C1000E
:100670007F2B3C083E02031D592B3D083F02031807
:10068000472BC0013F083D02C100A017582B3D0871
:100690003F02031D4F2BC001C101A017582B3F087B
:1006A0003D020318582BC0013D083F02C100A013B2
:1006B0007F2B3E083C0203187F2BA0133D083F020E
:1006C00003186C2B3C083E02C20001304202C000FD
:1006D0003D083F02C1007F2B3D083F02031D752BE3
:1006E0003C083E02C000C1017F2B3F083D020318B9
:1006F0007F2B3C083E02C0003D083F02C1000800BD
:10070000C1003D08FF3CC2003F08420203188D2B88
:100710003C083E07013EC000902B3C083E07C0004D
:100720003D083F07C1000800BE003C08C1003D086D
:100730000F39C2003E08DE234308BE000800BE0099
:100740003C08C1003D0E0F39C2003E08DE234308BD
:10075000BE003C08C1003D080F39C2003E08DE2340
:100760004308BE000800BE003D08C1006430C2005E
:100770008A244308BF003F08BD003C08C1003D0873
:10078000C4000A30C50099244608C3004308C200CB
:100790003E08DE234308BE003D08C1000A30C20007
:1007A0008A244308C0004008BD003C08C1003D0841
:1007B000C2003E08DE234308BE000800C300C20892
:1007C000031DEA2BC3080319E92B4308A100410AC2
:1007D0000620FC2B0A3042020318F42B4208303E5C
:1007E000A100410A0620FA2B0A304202413EA10034
:1007F000410A06203030C3000800BC003C08BD00A0
:100800006430BE006430122CBC003C08BD00643073
:10081000BE001430122CBC003C08BD006430BE0089
:100820000130122CBF00FF30C0003E08C2003D085E
:10083000C1001730400703181A2CC10B192CC20B2A
:10084000172CBF0B152C0800BF003F08C000C008C4
:10085000031D2B2C2F2C0A303024C003272C08001A
:10086000C600F430C700FC30C80046084707031C28
:10087000003448070318392C080063000800BD0045
:100880003C08831603139B0083123D0883169A00CD
:100890001C158B1355309D00AA309D009C149C188C
:1008A0004F2C1C118B1783120800BD003C088316C7
:1008B00003139B001C141A088312BD0008006D2C42
:1008C000702C702C702C702CC60046080F39C70095
:1008D0002508F0394704A5006D2C2508860008007E
:1008E000240885000800A60026080F39A700230861
:1008F000F0392704A300842C842C842C842C842C91
:10090000872C872C872C872C230866000800220858
:1009100065000800C2080319962C4208410203181A
:10092000922C962C42084102C1008D2C4108C30034
:100930000800C701C5080319A72C4508440203187D
:10094000A22CA72C45084402C400C70A9D2C4708C6
:10095000C6000800C3014108003C031CB02CB62CA3
:100960004008C30701304102C100AB2C4308C2005C
:0809700008000430A10008009A
:02400E00613F10
:00000001FF
